 pwm

 Timestamp is 4da293d5 (Mon Apr 11 17:38:29 2011)

 Preferred load address is 10000000

 Start         Length     Name                   Class
 0001:00000000 00000028H .rdata                  CODE
 0001:00000028 00000020H .rdata$debug            CODE
 0001:00000048 00000a68H .text                   CODE
 0001:00000ab0 00000004H .xdata                  CODE
 0001:00000ab4 0000003cH .idata$2                CODE
 0001:00000af0 00000014H .idata$3                CODE
 0001:00000b04 00000058H .idata$4                CODE
 0001:00000b5c 00000060H .idata$6                CODE
 0001:00000bc0 000000ecH .edata                  CODE
 0002:00000000 00000058H .idata$5                DATA
 0002:00000058 00000008H .data                   DATA
 0003:00000000 000000c8H .pdata                  DATA

  Address         Publics by Value              Rva+Base       Lib:Object

 0000:00000000       ___safe_se_handler_count   00000000     <absolute>
 0000:00000000       ___safe_se_handler_table   00000000     <absolute>
 0001:0000001c       ??_C@_1M@EENNDIOJ@?$AAI?$AAn?$AAd?$AAe?$AAx?$AA?$AA@ 1000101c     pwm_mx25_topaz_v1:pwmpdd.obj
 0001:00000048       BSPGetPWMClockSource       10001048 f   bsppwm.obj
 0001:00000050       BSPPwmSetClockGatingMode   10001050 f   bsppwm.obj
 0001:000000b0       BSPPwmIomuxSetPin          100010b0 f   bsppwm.obj
 0001:0000011c       BSPPwmGetBaseAddress       1000111c f   bsppwm.obj
 0001:0000016c       PWM_Init                   1000116c f   pwm_mx25_topaz_v1:pwmmdd.obj
 0001:00000170       PWM_Deinit                 10001170 f   pwm_mx25_topaz_v1:pwmmdd.obj
 0001:00000180       PWM_Open                   10001180 f   pwm_mx25_topaz_v1:pwmmdd.obj
 0001:000001f4       PWM_Close                  100011f4 f   pwm_mx25_topaz_v1:pwmmdd.obj
 0001:00000270       PWM_PowerDown              10001270 f   pwm_mx25_topaz_v1:pwmmdd.obj
 0001:00000274       PWM_PowerUp                10001274 f   pwm_mx25_topaz_v1:pwmmdd.obj
 0001:00000278       PWM_Read                   10001278 f   pwm_mx25_topaz_v1:pwmmdd.obj
 0001:00000294       PWM_Write                  10001294 f   pwm_mx25_topaz_v1:pwmmdd.obj
 0001:000002b4       PWM_IOControl              100012b4 f   pwm_mx25_topaz_v1:pwmmdd.obj
 0001:00000490       PWM_DllEntry               10001490 f   pwm_mx25_topaz_v1:pwmmdd.obj
 0001:000004a4       PwmDeinit                  100014a4 f   pwm_mx25_topaz_v1:pwmpdd.obj
 0001:000004e4       PwmReadRegister            100014e4 f   pwm_mx25_topaz_v1:pwmpdd.obj
 0001:00000560       SetPwmPower                10001560 f   pwm_mx25_topaz_v1:pwmpdd.obj
 0001:00000594       PwmGetRegistryValues       10001594 f   pwm_mx25_topaz_v1:pwmpdd.obj
 0001:000005fc       PwmOpen                    100015fc f   pwm_mx25_topaz_v1:pwmpdd.obj
 0001:00000600       PwmPlaySample              10001600 f   pwm_mx25_topaz_v1:pwmpdd.obj
 0001:0000077c       PwmInitialize              1000177c f   pwm_mx25_topaz_v1:pwmpdd.obj
 0001:00000858       PwmReset                   10001858 f   pwm_mx25_topaz_v1:pwmpdd.obj
 0001:000008d4       LocalAlloc                 100018d4 f   coredll:COREDLL.dll
 0001:000008e4       LocalFree                  100018e4 f   coredll:COREDLL.dll
 0001:000008f4       SetLastError               100018f4 f   coredll:COREDLL.dll
 0001:00000904       DisableThreadLibraryCalls  10001904 f   coredll:COREDLL.dll
 0001:00000914       DeleteCriticalSection      10001914 f   coredll:COREDLL.dll
 0001:00000924       LeaveCriticalSection       10001924 f   coredll:COREDLL.dll
 0001:00000934       EnterCriticalSection       10001934 f   coredll:COREDLL.dll
 0001:00000944       RegQueryValueExW           10001944 f   coredll:COREDLL.dll
 0001:00000954       OpenDeviceKey              10001954 f   coredll:COREDLL.dll
 0001:00000964       GetTickCount               10001964 f   coredll:COREDLL.dll
 0001:00000974       InitializeCriticalSection  10001974 f   coredll:COREDLL.dll
 0001:00000984       MmUnmapIoSpace             10001984 f   ceddk:CEDDK.dll
 0001:00000994       MmMapIoSpace               10001994 f   ceddk:CEDDK.dll
 0001:000009a4       DDKClockSetGatingMode      100019a4 f   cspddk:CSPDDK.dll
 0001:000009b4       DDKIomuxSetPinMux          100019b4 f   cspddk:CSPDDK.dll
 0001:000009c4       DDKClockGetFreq            100019c4 f   cspddk:CSPDDK.dll
 0001:000009d4       __GSHandlerCheckCommon     100019d4 f   corelib0:gshandler.obj
 0001:00000a0c       __GSHandlerCheck           10001a0c f   corelib0:gshandler.obj
 0001:00000a2c       __security_check_cookie    10001a2c f   corelib0:armsecgs.obj
 0001:00000a3c       __gsfailure                10001a3c     corelib0:armsecgs.obj
 0001:00000a80       memset                     10001a80 f   corelib1:COREDLL.dll
 0001:00000a90       __rt_udiv                  10001a90 f   corelib1:COREDLL.dll
 0001:00000aa0       __report_gsfailure         10001aa0 f   corelib1:COREDLL.dll
 0001:00000ab4       __IMPORT_DESCRIPTOR_COREDLL 10001ab4     coredll:COREDLL.dll
 0001:00000ac8       __IMPORT_DESCRIPTOR_CEDDK  10001ac8     ceddk:CEDDK.dll
 0001:00000adc       __IMPORT_DESCRIPTOR_CSPDDK 10001adc     cspddk:CSPDDK.dll
 0001:00000af0       __NULL_IMPORT_DESCRIPTOR   10001af0     coredll:COREDLL.dll
 0002:00000000       __imp_MmUnmapIoSpace       10002000     ceddk:CEDDK.dll
 0002:00000004       __imp_MmMapIoSpace         10002004     ceddk:CEDDK.dll
 0002:00000008       \177CEDDK_NULL_THUNK_DATA  10002008     ceddk:CEDDK.dll
 0002:0000000c       __imp_DisableThreadLibraryCalls 1000200c     coredll:COREDLL.dll
 0002:00000010       __imp_DeleteCriticalSection 10002010     coredll:COREDLL.dll
 0002:00000014       __imp_LeaveCriticalSection 10002014     coredll:COREDLL.dll
 0002:00000018       __imp_EnterCriticalSection 10002018     coredll:COREDLL.dll
 0002:0000001c       __imp_SetLastError         1000201c     coredll:COREDLL.dll
 0002:00000020       __imp_OpenDeviceKey        10002020     coredll:COREDLL.dll
 0002:00000024       __imp_GetTickCount         10002024     coredll:COREDLL.dll
 0002:00000028       __imp_InitializeCriticalSection 10002028     coredll:COREDLL.dll
 0002:0000002c       __imp_LocalFree            1000202c     coredll:COREDLL.dll
 0002:00000030       __imp_RegQueryValueExW     10002030     coredll:COREDLL.dll
 0002:00000034       __imp_LocalAlloc           10002034     coredll:COREDLL.dll
 0002:00000038       __imp___rt_udiv            10002038     corelib1:COREDLL.dll
 0002:0000003c       __imp_memset               1000203c     corelib1:COREDLL.dll
 0002:00000040       __imp___report_gsfailure   10002040     corelib1:COREDLL.dll
 0002:00000044       \177COREDLL_NULL_THUNK_DATA 10002044     coredll:COREDLL.dll
 0002:00000048       __imp_DDKIomuxSetPinMux    10002048     cspddk:CSPDDK.dll
 0002:0000004c       __imp_DDKClockSetGatingMode 1000204c     cspddk:CSPDDK.dll
 0002:00000050       __imp_DDKClockGetFreq      10002050     cspddk:CSPDDK.dll
 0002:00000054       \177CSPDDK_NULL_THUNK_DATA 10002054     cspddk:CSPDDK.dll
 0002:00000058       __security_cookie          10002058     corelib0:seccinit.obj
 0002:0000005c       __security_cookie_complement 1000205c     corelib0:seccinit.obj

 entry point at        0001:00000490

 Static symbols

